:020000040800F2
:1000000000000220E5110008390800083B0800083C
:100010003D0800083F0800084108000800000000F3
:10002000000000000000000000000000430800087D
:1000300045080008000000004708000849080008BB
:100040003512000835120008351200083512000874
:100050003512000835120008351200083512000864
:100060003512000835120008351200083512000854
:100070003512000835120008351200083512000844
:100080003512000835120008351200080000000083
:100090000000000000000000000000003512000811
:1000A0003512000835120008351200083512000814
:1000B0003512000835120008351200083512000804
:1000C00035120008351200083512000835120008F4
:1000D0003512000835120008351200080000000033
:1000E0003512000835120008351200080000000023
:1000F00000000000000000000000000035120008B1
:100100000000000035120008351200083512000802
:1001100000000000000000000000000000000000DF
:100120003512000835120008351200083512000893
:100130003512000800000000000000000000000070
:100140000000000000000000000000003512000860
:100150003512000835120008351200083512000863
:1001600035120008351200080000000000000000F1
:10017000000000000000000000000000000000007F
:100180000000000035120008000000000000000020
:080190003512000835120008C9
:100198000348044B834202D0034B03B1184770470E
:1001A8003C0400203C040020000000000548064BE9
:1001B8001B1AD90F01EBA301491002D0034B03B15D
:1001C800184770473C0400203C0400200000000051
:1001D80010B5064C237843B9FFF7DAFF044B13B187
:1001E8000448AFF300800123237010BD3C040020B5
:1001F800000000004C12000808B5044B1BB104496C
:100208000448AFF30080BDE80840CFE700000000D5
:10021800400400204C12000853B94AB9002908BF0D
:1002280000281CBF4FF0FF314FF0FF3000F06AB9D3
:10023800ADF1080C6DE904CE00F006F8DDF804E035
:10024800DDE9022304B070472DE9F047089D0C460C
:10025800002B4ED194468C458646B2FA82F262D97A
:100268004AB1C2F12003914020FA03F30CFA02FCD0
:10027800194300FA02FE4FEA1C471FFA8CF6B1FB3D
:10028800F7F44FEA1E4307FB141143EA014304FB4A
:1002980006F199420AD91CEB030304F1FF3080F000
:1002A8001381994240F21081023C6344591A1FFAA3
:1002B8008EF3B1FBF7F007FB101143EA014300FB93
:1002C80006F69E420AD91CEB030300F1FF3180F0C9
:1002D800FD809E4240F2FA80634402389B1B40EA4C
:1002E800044000211DB1D3400022C5E90032BDE819
:1002F800F0878B4205D90DB1C5E9000100210846F8
:10030800F5E7B3FA83F1002946D1A34202D390421C
:10031800C0F0F180861A64EB03030120002DE6D0BB
:10032800C5E90063E3E7002A40F09180A1EB0C04E3
:100338004FEA1C481FFA8CF70121B4FBF8F64FEA84
:100348001E4308FB164443EA044307FB06F09842A1
:1003580008D91CEB030306F1FF3402D2984200F2DD
:10036800CE8026461C1A1FFA8EF3B4FBF8F008FB61
:10037800104443EA044300FB07F79F4208D91CEBEB
:10038800030300F1FF3402D29F4200F2B1802046FD
:10039800DB1B40EA0640A5E7C1F120068B4022FAA4
:1003A80006F71F4320FA06FC04FA01F343EA0C039C
:1003B800F44000FA01F8380C4FEA1349B4FBF0FE98
:1003C8001FFA87FC00FB1E4449EA04440EFB0CF9A3
:1003D800A14502FA01F20AD93C190EF1FF3A80F060
:1003E8008580A14540F28280AEF1020E3C44A4EB28
:1003F80009041FFA83F9B4FBF0F300FB134449EA3C
:10040800044403FB0CFCA44507D93C1903F1FF3055
:1004180068D2A44566D9023B3C4443EA0E40A0FB9F
:100428000293A4EB0C049C42CE469C4652D34FD078
:1004380055B1B8EB0E0364EB0C0404FA06F6CB4096
:10044800CC401E43C5E900640021BDE8F087C2F135
:10045800200320FA03F10CFA02FC24FA03F3944077
:100468000C434FEA1C4800FA02FE1FFA8CF7B3FB54
:10047800F8F008FB1031230C43EA014300FB07F1B5
:10048800994208D91CEB030300F1FF362CD299429C
:100498002AD9023863445B1AA4B2B3FBF8F108FB0B
:1004A800113344EA034401FB07F3A34208D91CEBC8
:1004B800040401F1FF3613D2A34211D9023964446E
:1004C800E41A41EA004138E70446EFE6084605E742
:1004D800C845ADD2B9EB020E63EB070C0138A7E7AC
:1004E8003146EDE7034698E73046D4E7D6467EE73F
:1004F800634402384CE70646234608460EE7023EA8
:1005080063442FE7704700BF002301461A46184688
:1005180000F08CB838B5084B084D5B1B9C1007D011
:10052800043B1D44013C55F804399847002CF9D187
:10053800BDE8384000F08CBE8C1200088812000814
:1005480070B50D4E0D4D761BB61006D0002455F82B
:10055800043B01349847A642F9D1094E094D761B50
:1005680000F070FEB61006D0002455F8043B0134A4
:100578009847A642F9D170BD801200088012000881
:100588008812000880120008830730B548D0541E2E
:10059800002A3FD0CAB2034601E0013C3AD303F82F
:1005A800012B9D07F9D1032C2DD9CDB245EA05259C
:1005B8000F2C45EA054536D9A4F1100222F00F0C9C
:1005C80003F1200EE6444FEA121C03F1100242E93F
:1005D800045542E9025510327245F8D10CF1010276
:1005E80014F00C0F03EB021204F00F0C13D0ACF153
:1005F800040323F003030433134442F8045B9342D7
:10060800FBD10CF003042CB1CAB21C4403F8012B33
:100618009C42FBD130BD64461346002CF4D1F9E767
:1006280003461446BFE71A46A446E0E770B4184CE0
:100638002568D5F848411CB365681F2D25DC38B9F5
:10064800AB1C0135656044F82310002070BC70476E
:1006580004EB850C0228CCF88820D4F888614FF088
:10066800010202FA05F246EA0206C4F88861CCF8EB
:100678000831E5D1D4F88C311343C4F88C31DFE765
:1006880005F5A674C5F84841D6E74FF0FF30DDE719
:100698006412000808B54FF40051034800F094FABA
:1006A800322000F025F9F6E70008024070B588B05E
:1006B80000240394049405940694079400941C4B16
:1006C8001A6B42F004021A631A6B02F004020092D9
:1006D800009A01941A6B42F080021A631A6B02F0B6
:1006E80080020192019A02941A6B42F001021A6385
:1006F8001B6B03F001030293029B0E4E22464FF43C
:100708000051304600F05AFA4FF400530393012584
:1007180004950594069403A9304600F067F90395FB
:100728000494059403A9044800F060F908B070BD6A
:1007380000380240000802400000024072B6FEE79E
:1007480000B595B03022002108A8FFF71DFF00234F
:100758000393049305930693079301931F4A116C1F
:1007680041F080511164126C02F080520192019A9A
:1007780002931B4B1A6842F440421A601B6803F448
:1007880040430293029B012308934FF4803309935B
:1007980002230E934FF480020F920C2210926022D3
:1007A800119212930423139308A800F017FA88B93A
:1007B8000F23039302230493002305934FF48052DD
:1007C80006920793032103A800F058FC20B915B03E
:1007D8005DF804FBFFF7B2FFFFF7B0FF00380240F7
:1007E8000070004008B500F057F8FFF7A9FFFFF7C1
:1007F8005DFFFFF74FFFFEE782B0002100910B4B32
:100808005A6C42F480425A645A6C02F48042009254
:10081800009A01911A6C42F080521A641B6C03F022
:1008280080530193019B02B0704700BF003802401B
:10083800FEE7FEE7FEE7FEE7FEE770477047704712
:1008480008B500F043F808BD7047000010B504462D
:100858000E4B1A784FF47A73B3FBF2F30C4A106814
:10086800B0FBF3F000F0AEF868B90F2C01D9012005
:100878000AE0002221464FF0FF3000F093F8054BC4
:100888001C60002000E0012010BD00BF34040020DF
:10089800300400203804002008B50B4B1A6842F4D5
:1008A80000721A601A6842F480621A601A6842F488
:1008B80080721A60032000F063F80F20FFF7C6FF6C
:1008C800FFF79AFF002008BD003C0240034A116868
:1008D800034B1B780B441360704700BF580400207B
:1008E80034040020014B1868704700BF58040020EA
:1008F80038B50446FFF7F6FF0546B4F1FF3F02D0CE
:10090800044B1B781C44FFF7EDFF401BA042FAD3B1
:1009180038BD00BF34040020002808DB0901C9B233
:1009280000F1604000F5614080F80013704700F066
:100938000F000901C9B2014B1954704714ED00E0CA
:1009480000B500F00700C0F1070CBCF1040F28BF88
:100958004FF0040C031D062B0FD9C31E4FF0FF3EAA
:100968000EFA0CF021EA000199400EFA03FE22EA81
:100978000E0241EA02005DF804FB0023EEE70000E6
:10098800074AD36823F4E0631B041B0C000200F43D
:10099800E060034343F0BF6343F40033D360704720
:1009A80000ED00E010B50446054BD868C0F30220FE
:1009B800FFF7C6FF01462046FFF7AEFF10BD00BF98
:1009C80000ED00E00138B0F1807F0BD24FF0E0235A
:1009D8005861054AF02182F8231000209861072207
:1009E8001A6170470120704700ED00E000230F2BCB
:1009F80000F2DA8030B583B068E085684FEA430ECC
:100A0800032404FA0EF425EA0405CC6804FA0EF46B
:100A18002C438460446824EA02044A68C2F3001242
:100A28009A40224342605FE0DC08083450F82420F2
:100A380003F00705AD004FF00F0E0EFA05FE22EA8F
:100A48000E0E0A69AA4042EA0E0240F824205FE02E
:100A5800042200E0002202FA0EF22A430234534D27
:100A680045F82420524A94686FEA0C0224EA0C05DF
:100A7800D1F804E01EF4801F01D04CEA04054C4C68
:100A8800A560E46802EA0405D1F804E01EF4001F3A
:100A980001D04CEA0405464CE560646802EA0405A6
:100AA800D1F804E01EF4003F01D04CEA0405404CA4
:100AB8006560246822404D6815F4803F01D04CEAF7
:100AC80004023B4C226001330F2B6BD801229A4061
:100AD8000C6804EA020C32EA0404F4D14C6804F00D
:100AE8000304013C012C88D94A6802F00302032A56
:100AF80009D0C4685D000322AA4024EA02048A6877
:100B0800AA402243C2604A6802F00302022A8BD03C
:100B180004684FEA430E032202FA0EF224EA0204A2
:100B28004A6802F0030202FA0EF2224302604A689F
:100B380012F4403FC7D0002201921E4A546C44F47C
:100B480080445464526C02F480420192019A9C08D9
:100B5800A51C164A52F8255003F0030E4FEA8E0ED4
:100B68000F2202FA0EF225EA0205134A90423FF4D8
:100B780071AF02F5806290420ED002F58062904219
:100B88000CD002F5806290420AD002F58062904251
:100B98003FF45EAF07225EE701225CE702225AE7D4
:100BA800032258E703B030BD704700BF003801404A
:100BB800003C014000380240000002400AB1816157
:100BC8007047090481617047436901EA030221EA19
:100BD800030141EA0241816170470000002800F0EA
:100BE800E08170B582B00446036813F0010F3BD072
:100BF8009F4B9B6803F00C03042B2CD09C4B9B68E9
:100C080003F00C03082B21D06368B3F5803F4FD065
:100C1800B3F5A02F52D0964B1A6822F480321A608E
:100C28001A6822F480221A606368002B50D0FFF7FC
:100C380059FE05468E4B1B6813F4003F14D1FFF78D
:100C480051FE401B6428F5D90320B1E1884B5B684D
:100C580013F4800FD8D0864B1B6813F4003F03D0E1
:100C68006368002B00F09F81236813F0020F54D0B3
:100C78007F4B9B6813F00C0F3ED07D4B9B6803F0B5
:100C88000C03082B33D0E368002B68D0794B012282
:100C98001A60FFF727FE0546754B1B6813F0020F15
:100CA80054D1FFF71FFE401B0228F5D903207FE12E
:100CB8006F4A136843F480331360B5E76C4B1A68C6
:100CC80042F480221A601A6842F480321A60ABE754
:100CD800FFF708FE0546664B1B6813F4003FC3D0B8
:100CE800FFF700FE401B6428F5D9032060E1604B44
:100CF8005B6813F4800FC6D15D4B1B6813F0020FBD
:100D080003D0E368012B40F05081594A136823F05F
:100D1800F803216943EAC1031360236813F0080F3D
:100D280042D063696BB3534B0122C3F8802EFFF79F
:100D3800D9FD05464E4B5B6F13F0020F34D1FFF718
:100D4800D1FD401B0228F5D9032031E1484A136838
:100D580023F0F803216943EAC1031360DDE7454B3B
:100D680000221A60FFF7BEFD0546414B1B6813F0D1
:100D7800020FD2D0FFF7B6FD401B0228F5D9032099
:100D880016E13C4B0022C3F8802EFFF7ABFD054669
:100D9800374B5B6F13F0020F06D0FFF7A3FD401B24
:100DA8000228F5D9032003E1236813F0040F77D054
:100DB8002F4B1B6C13F0805F33D1002301932C4B16
:100DC8001A6C42F080521A641B6C03F08053019332
:100DD800019B0125284B1B6813F4807F23D0A3684F
:100DE800012B34D0052B38D0214B1A6F22F0010289
:100DF8001A671A6F22F004021A67A368002B3DD005
:100E0800FFF770FD06461A4B1B6F13F0020F46D111
:100E1800FFF768FD801B41F288339842F3D903201D
:100E2800C6E00025D6E7144A136843F480731360BC
:100E3800FFF758FD0646104B1B6813F4807FCED190
:100E4800FFF750FD801B0228F5D90320B0E0084ABF
:100E5800136F43F001031367CFE7054B1A6F42F096
:100E680004021A671A6F42F001021A67C5E700BF49
:100E7800003802400000474200700040FFF732FD92
:100E88000646524B1B6F13F0020F08D0FFF72AFDDE
:100E9800801B41F288339842F3D9032088E0EDB9EA
:100EA800A369002B00F08380484A926802F00C0284
:100EB800082A51D0022B17D0454B00221A66FFF79B
:100EC80011FD0446414B1B6813F0007F42D0FFF729
:100ED80009FD001B0228F5D9032069E03B4A136C81
:100EE80023F080531364DBE7394B00221A66FFF7BF
:100EF800F9FC0546354B1B6813F0007F06D0FFF759
:100F0800F1FC401B0228F5D9032051E0E369226A6D
:100F18001343626A43EA8213A26A5208013A43EA17
:100F28000243E26A43EA0263284A5360284B0122DB
:100F38001A66FFF7D7FC0446244B1B6813F0007FA2
:100F480006D1FFF7CFFC001B0228F5D903202FE0BC
:100F580000202DE000202BE0012B2BD01B4B5B68E1
:100F680003F48001E269914226D103F03F02216A2D
:100F78008A4223D1616A47F6C0721A40B2EB811FD8
:100F88001ED103F44031A26A5208013AB1EB024F74
:100F980018D103F07063E26AB3EB026F14D100203A
:100FA80006E001207047012002E0012000E0002057
:100FB80002B070BD0120FBE70120F9E70120F7E747
:100FC8000120F5E70120F3E70120F1E700380240AE
:100FD8000000474208B5264B9B6803F00C03042B1E
:100FE80041D0082B41D1224B5A6802F03F025B687E
:100FF80013F4800F12D01E4B5968C1F388111D4895
:101008000023A1FB0001FFF707F9194B5B68C3F345
:10101800014301335B00B0FBF3F027E0144B586841
:10102800C0F388104FEA401CBCEB000C6EEB0E0EB0
:101038004FEA8E1343EA9C634FEA8C11B1EB0C0123
:1010480063EB0E03DB0043EA5173C90011EB000C9C
:1010580043F10003990200234FEA8C2041EA9C5196
:10106800FFF7DAF8D1E7034800E0034808BD00BFFE
:101078000038024040787D010024F400002800F088
:101088009B8070B50D4604464F4B1B6803F0070361
:101098008B4208D2CBB24C4A1370136803F0070393
:1010A8008B4240F08B80236813F0020F17D013F0A7
:1010B800040F04D0454A936843F4E05393602368CF
:1010C80013F0080F04D0414A936843F460439360D7
:1010D8003E4A936823F0F003A1680B4393602368AA
:1010E80013F0010F32D06368012B21D09A1E012A18
:1010F80025D9364A126812F0020F61D033498A683E
:1011080022F0030213438B60FFF7ECFB06462F4BDC
:101118009B6803F00C036268B3EB820F16D0FFF7ED
:10112800E1FB801B41F288339842F0D9032042E06A
:10113800264A126812F4003FE0D101203BE0234A1E
:10114800126812F0007FD9D1012034E01E4B1B68D1
:1011580003F00703AB4207D9EAB21B4B1A701B68AE
:1011680003F00703AB422DD1236813F0040F06D018
:10117800164A936823F4E053E1680B4393602368AD
:1011880013F0080F07D0114A936823F460432169CC
:1011980043EAC1039360FFF71DFF0C4B9B68C3F341
:1011A80003130B4AD35CD8400A4B18600A4B1868E3
:1011B800FFF74CFB002070BD012070470120FAE7C3
:1011C8000120F8E70120F6E7003C02400038024021
:1011D800681200083004002038040020DFF834D0FA
:1011E8000D480E490E4A002302E0D458C450043377
:1011F800C4188C42F9D30B4A0B4C002301E013604E
:101208000432A242FBD3FFF71FFBFFF799F9FFF760
:10121800E9FA704700000220000000203C0400208A
:101228008C1200083C0400205C040020FEE700004B
:10123800024B13B10248FFF767B97047000000007E
:101248001D050008F8B500BFF8BC08BC9E467047ED
:0C125800F8B500BFF8BC08BC9E4670470B
:101264000800002000000000000000000102030448
:041274000607080958
:08127800D8EFFF7F0100000028
:08128000391200080102000808
:04128800D901000880
:10128C00080000200000000000000000F402002014
:10129C005C030020C40300200000000000000000DC
:1012AC000000000000000000000000000000000032
:1012BC000000000000000000000000000000000022
:1012CC000000000000000000000000000000000012
:1012DC000000000000000000000000000000000002
:1012EC0000000000000000000000000000000000F2
:1012FC0000000000000000000000000000000000E2
:10130C0000000000000000000000000000000000D1
:10131C0000000000000000000000000000000000C1
:10132C0000000000000000000000000000000000B1
:10133C0001000000000000000E33CDAB34126DE64E
:10134C00ECDE05000B0000000000000000000000B7
:10135C000000000000000000000000000000000081
:10136C000000000000000000000000000000000071
:10137C000000000000000000000000000000000061
:10138C000000000000000000000000000000000051
:0C16BC000024F4000100000010000000F9
:04000005080011E5F9
:00000001FF
